:020000040000FA
:04080000E7EF07F027
:1008100003B213EF05F0F2B42EEF05F09EB036EF01
:1008200005F09EB23EEF05F0F2A81AEF04F0F2B226
:1008300025EF04F0F2A620EF04F0F2B022EF04F06E
:1008400096EF07F0F296F290FF00CD90F2929EA004
:100850002FEF04F00101533F2FEF04F0542BAEC1F2
:10086000B2F1AFC1B3F1B0C1B4F1B1C1B5F1AAC138
:10087000AEF1ABC1AFF1ACC1B0F1ADC1B1F1A6C148
:10088000AAF1A7C1ABF1A8C1ACF1A9C1ADF1A2C158
:10089000A6F1A3C1A7F1A4C1A8F1A5C1A9F19EC168
:1008A000A2F19FC1A3F1A0C1A4F1A1C1A5F19AC178
:1008B0009EF19BC19FF19CC1A0F19DC1A1F196C188
:1008C0009AF197C19BF198C19CF199C19DF1CECF4E
:1008D00096F1CFCF97F153C198F154C199F1CF6AF6
:1008E000CE6A0101536B546B9E90CD800FBC0F8E6E
:1008F0000FBA7EEF04F00F8A96EF07F00F8C0FBE51
:10090000BAEF04F096C19AF197C19BF198C19CF19E
:1009100099C19DF19AC19EF19BC19FF19CC1A0F12B
:100920009DC1A1F19EC1A2F19FC1A3F1A0C1A4F1FB
:10093000A1C1A5F1A2C1A6F1A3C1A7F1A4C1A8F1CB
:10094000A5C1A9F1A6C1AAF1A7C1ABF1A8C1ACF19B
:10095000A9C1ADF1AAC1AEF1ABC1AFF1ACC1B0F16B
:10096000ADC1B1F1AEC1B2F1AFC1B3F1B0C1B4F13B
:10097000B1C1B5F101015E6B5F6B606B616B96514C
:100980005E2797515F2398516023995161239A51B3
:100990005E279B515F239C5160239D5161239E5193
:1009A0005E279F515F23A0516023A1516123A25173
:1009B0005E27A3515F23A4516023A5516123A65153
:1009C0005E27A7515F23A8516023A9516123AA5133
:1009D0005E27AB515F23AC516023AD516123AE5113
:1009E0005E27AF515F23B0516023B1516123B251F3
:1009F0005E27B3515F23B4516023B5516123D89072
:100A00000101613360335F335E33D890010161339C
:100A100060335F335E33D8900101613360335F33FD
:100A20005E3396EF07F00392030103EE00F080516E
:100A30007F0BE92604C0EFFF802B8151805D700B96
:100A4000D8A48B8200008051815D700BD8A48B925A
:100A500081518019D8B4079096EF07F0F294010104
:100A6000453F96EF07F0462B96EF07F09E90010169
:100A7000533F96EF07F0542B96EF07F09E92040039
:100A800062A143EF05F0077C07AC5EEF05F0C2748E
:100A9000C2B458EF05F0C3CFB3F5C4CFB4F5050128
:100AA000D890B433B333D890B433B3335FEF05F099
:100AB000C3CF55F1C4CF56F15FEF05F0C28207B442
:100AC000CCEF05F047C14BF148C14CF149C14DF1A4
:100AD0004AC14EF15EC162F15FC163F160C164F170
:100AE00061C165F196C1B6F197C1B7F198C1B8F18E
:100AF00099C1B9F19AC1BAF19BC1BBF19CC1BCF1DA
:100B00009DC1BDF19EC1BEF19FC1BFF1A0C1C0F1A9
:100B1000A1C1C1F1A2C1C2F1A3C1C3F1A4C1C4F179
:100B2000A5C1C5F1A6C1C6F1A7C1C7F1A8C1C8F149
:100B3000A9C1C9F1AAC1CAF1ABC1CBF1ACC1CCF119
:100B4000ADC1CDF1AEC1CEF1AFC1CFF1B0C1D0F1E9
:100B5000B1C1D1F1B2C1D2F1B3C1D3F1B4C1D4F1B9
:100B6000B5C1D5F1B3C5B5F5B4C5B6F5B5C5B7F5DD
:100B7000B6C5B8F5010155515B2756515C23E86AAB
:100B80005D230E2ECCEF05F05CC157F15DC158F12D
:100B90005B6B5C6B5D6B078E0201002F96EF07F0BD
:100BA0003C0E006F00C10CF101C10DF102C10EF14C
:100BB00003C10FF104C110F105C111F106C112F119
:100BC00007C113F108C114F109C115F10AC116F1E9
:100BD0000BC117F134C135F105012F51000AD8B40A
:100BE00095EF06F005012F51010AD8B41FEF06F06A
:100BF00005012F51020AD8B460EF06F005012F510C
:100C0000030AD8B460EF06F005012F51040AD8B4E6
:100C100060EF06F005012F51050AD8B460EF06F029
:100C200005012F51060AD8B460EF06F005012F51D7
:100C3000070AD8B460EF06F02F6B95EF06F00501B8
:100C400053672AEF06F054672AEF06F055672AEF3C
:100C500006F056672EEF06F095EF06F057C500F147
:100C600058C501F159C502F15AC503F10101010E40
:100C7000046F000E056F000E066F000E076F20EC6C
:100C800022F000C157F501C158F502C159F503C161
:100C90005AF5006753EF06F0016753EF06F002675D
:100CA00053EF06F0036795EF06F053C557F554C5AB
:100CB00058F555C559F556C55AF50F8895EF06F004
:100CC0000501306766EF06F095EF06F00FBE7BEF8B
:100CD00006F010A080EF06F00101476777EF06F0FD
:100CE000486777EF06F0496777EF06F04A677BEFD2
:100CF00006F080EF06F007AE80EF06F092EF06F008
:100D00000501312F95EF06F03C0E316F302F95EF36
:100D100006F00101000E626FE00E636FA50E646FB6
:100D2000010E656F0501306B0F880501626B33B7EB
:100D30009BEF06F062810CC100F10DC101F10EC103
:100D400002F10FC103F110C104F111C105F112C18B
:100D500006F113C107F114C108F115C109F116C15B
:100D60000AF117C10BF135C134F100C10CF101C119
:100D70000DF102C10EF103C10FF104C110F105C163
:100D800011F106C112F107C113F108C114F109C133
:100D900015F10AC116F10BC117F134C135F101018A
:100DA0008A67DAEF06F08B67DAEF06F08C67DAEF26
:100DB00006F08D67DEEF06F00EEF07F08EC100F152
:100DC0008FC101F190C102F191C103F10101010E46
:100DD000046F000E056F000E066F000E076F20EC0B
:100DE00022F000C18EF101C18FF102C190F103C167
:100DF00091F1006703EF07F0016703EF07F0026767
:100E000003EF07F003670EEF07F08AC18EF18BC185
:100E10008FF18CC190F18DC191F10F80D57ED5BE3F
:100E200069D0D6CF47F1D7CF48F145C149F1E86A3B
:100E3000E8CF4AF1109047C100F148C101F149C122
:100E400002F14AC103F101010A0E046F000E056FA1
:100E5000000E066F000E076F20EC22F000AF10802E
:100E6000010154A740EF07F00F9A0F9C0F9E01015C
:100E7000000E5E6F600E5F6F3D0E606F080E616F5B
:100E8000010147BF50EF07F0486750EF07F049678F
:100E900050EF07F04A6750EF07F0F28875EF07F060
:100EA000F2985E6B5F6B606B616B966B976B986B88
:100EB000996B9A6B9B6B9C6B9D6B9E6B9F6BA06BF6
:100EC000A16BA26BA36BA46BA56BA66BA76BA86BA6
:100ED000A96BAA6BAB6BAC6BAD6BAE6BAF6BB06B56
:100EE000B16BB26BB36BB46BB56BD76AD66A0101E9
:100EF000456B466B0CC100F10DC101F10EC102F151
:100F00000FC103F110C104F111C105F112C106F1C5
:100F100013C107F114C108F115C109F116C10AF195
:100F200017C10BF135C134F196EF07F002C0E0FFB5
:100F3000005001C0D8FF1000A6B29CEF07F00CC013
:100F4000A9FF0BC0A8FFA69EA69CA684F29E550EE4
:100F5000A76EAA0EA76EA682F28EA694A6B2AEEFD8
:100F600007F00C2A1200A96EA69EA69CA680A85087
:100F70000C2A120004012C0E826FA9EC0AF01BEC63
:100F800023F00C50B3EC07F0E8CF00F10C50B3ECB9
:100F900007F0E8CF01F101AFD3EF07F00101FF0E39
:100FA000026FFF0E036FBEEC22F02967DFEF07F040
:100FB0000401200E826FA9EC0AF0E4EF07F00401AF
:100FC0002D0E826FA9EC0AF0E8EC20F01200076AFF
:100FD0000F6A106A0F010D0EC16E860EC06E030EF1
:100FE000C26E0F01280E896E130E926E080E8A6E65
:100FF0008A6AF30E936E010E8B6E900E946EF18ED4
:10100000F19E0E6A01015B6B5C6B5D6B576B586BFD
:10101000F29A0101476B486B496B4A6B4B6B4C6B07
:101020004D6B4E6B4F6B506B516B526B456B466B00
:10103000D76AD66A0F01280ED56EF28A9D90B00E3F
:10104000CD6E01015E6B5F6B606B616B626B636B9E
:10105000646B656B666B676B686B696B536B546B2A
:10106000CF6ACE6A0F9A0F9C0F9E9D80760ECA6E35
:101070009D8202013C0E006FCC6A160EB3EC07F0A5
:10108000E8CF00F1170EB3EC07F0E8CF01F1180E2E
:10109000B3EC07F0E8CF02F1190EB3EC07F0E8CF9C
:1010A00003F1010103AF6FEF08F01BEC23F0160E04
:1010B0000C6E00C10BF09CEC07F0170E0C6E01C11A
:1010C0000BF09CEC07F0180E0C6E02C10BF09CECC0
:1010D00007F0190E0C6E03C10BF09CEC07F000C179
:1010E0008AF101C18BF102C18CF103C18DF100C104
:1010F0008EF101C18FF102C190F103C191F11A0E7D
:10110000B3EC07F0E8CF00F11B0EB3EC07F0E8CF2B
:1011100001F11C0EB3EC07F0E8CF02F11D0EB3ECA9
:1011200007F0E8CF03F1010103AFC5EF08F01BECB6
:1011300023F01A0E0C6E00C10BF09CEC07F01B0E96
:101140000C6E01C10BF09CEC07F01C0E0C6E02C182
:101150000BF09CEC07F01D0E0C6E03C10BF09CEC29
:1011600007F01A0EB3EC07F0E8CF00F11B0EB3EC5A
:1011700007F0E8CF01F11C0EB3EC07F0E8CF02F165
:101180001D0EB3EC07F0E8CF03F100C192F101C1ED
:1011900093F102C194F103C195F1240EAC6E900E4F
:1011A000AB6E240EAC6E080EB86E000EB06E1F0E45
:1011B000AF6E0401806B816B0F01900EAB6E0F015F
:1011C0009D8A0301806B816BC26B8B92ABEC29F023
:1011D0000BEC2BF08BEC27F0200EB3EC07F0E8CFF4
:1011E0002FF505012F51FF0AD8A4FEEF08F02F6B51
:1011F000200E0C6E2FC50BF09CEC07F00501010EC4
:10120000306F3C0E316F250EB3EC07F0E8CF00F1E4
:10121000260EB3EC07F0E8CF01F1270EB3EC07F090
:10122000E8CF02F1280EB3EC07F0E8CF03F101019B
:1012300003AF35EF09F01BEC23F0250E0C6E00C157
:101240000BF09CEC07F0260E0C6E01C10BF09CEC31
:1012500007F0270E0C6E02C10BF09CEC07F0280E75
:101260000C6E03C10BF09CEC07F000C153F501C1FB
:1012700054F502C155F503C156F500C157F501C13A
:1012800058F502C159F503C15AF5290EB3EC07F020
:10129000E8CF5BF505015C515B5DD8A05BC55CF5F3
:1012A00005012F51020A0EE181B862EF09F0050134
:1012B0005C2F5FEF09F05BC55CF562EF09F081BA66
:1012C0004AEF2BF0210EB3EC07F0E8CF00F1220E2D
:1012D000B3EC07F0E8CF01F1230EB3EC07F0E8CF51
:1012E00002F1240EB3EC07F0E8CF03F1010103AFE4
:1012F000A8EF09F01BEC23F0210E0C6E00C10BF0DF
:101300009CEC07F0220E0C6E01C10BF09CEC07F078
:10131000230E0C6E02C10BF09CEC07F0240E0C6E39
:1013200003C10BF09CEC07F0210EB3EC07F0E8CF03
:1013300000F1220EB3EC07F0E8CF01F1230EB3EC7D
:1013400007F0E8CF02F1240EB3EC07F0E8CF03F189
:1013500000C15DF501C15EF502C15FF503C160F535
:10136000C2EC26F084EC25F0D4EC24F005012F51DA
:10137000030A12E005012F51040A1DE005012F5157
:10138000050A24E005012F51060A32E005012F511C
:10139000070A38E00BEF0AF0ACC500F101010F0EAF
:1013A000001701010051000A36E001010051050A51
:1013B00032E008EF0AF0ACC500F101010F0E001792
:1013C00001010051000A27E008EF0AF00501AC51C5
:1013D000000A21E00501AC51150A1DE00501AC51E0
:1013E000300A19E00501AC51450A15E008EF0AF092
:1013F0000501AC51000A0FE00501AC51300A0BE0C9
:1014000008EF0AF00501AC51000A05E008EF0AF008
:1014100081BA4AEF2BF08A867FEC24F00790000116
:10142000F28EF28C07B069EF1FF00FB04AEF1AF09E
:101430000FB80EEF14F00301805181197F0BD8B45F
:1014400069EF1FF013EE00F081517F0BE126812B35
:10145000E7CFE8FFE00BD8B469EF1FF023EE82F08E
:10146000C2513F0BD926E7CFDFFFC22BDF50780AEE
:10147000D8A469EF1FF007808EC100F18FC101F180
:1014800090C102F191C103F10101040E046F000E3D
:10149000056F000E066F000E076F20EC22F000AF04
:1014A0005BEF0AF00101030E8E6F000E8F6F000ECE
:1014B000906F000E916F03018251720AD8B44AEF07
:1014C0001AF08251520AD8B44AEF1AF08251750AC2
:1014D000D8B44AEF1AF08251630AD8B425EF1CF051
:1014E0008251690AD8B405EF17F082517A0AD8B44C
:1014F00018EF18F08251490AD8B4A4EF16F08251BF
:10150000500AD8B4C2EF15F08251700AD8B405EF72
:1015100016F08251540AD8B430EF16F08251740A92
:10152000D8B476EF16F08251730AD8B47AEF19F076
:101530008251530AD8B4DFEF19F082514C0AD8B463
:101540004FEF0EF08251760AD8B4BDEF0AF05AEF91
:101550001CF0040114EE00F080517F0BE12682C4E0
:10156000E7FF802B120004010D0E826FA9EC0AF038
:101570000A0E826FA9EC0AF0120003018351300AAF
:10158000D8B4DEEF0AF003018351310AD8B415EF65
:101590000BF003018351320AD8B4EBEF0BF00301D7
:1015A0008351330AD8B4C1EF0CF003018351340ADC
:1015B000D8B467EF0DF0D8A45AEF1CF00401760EF2
:1015C000826FA9EC0AF00401300E826FA9EC0AF0D8
:1015D00004012C0E826FA9EC0AF089EC23F01BECBD
:1015E00023F000C600F101C601F1BEEC22F030C1CB
:1015F00082F40401300E8227A9EC0AF031C182F492
:101600000401300E8227A9EC0AF032C182F40401F1
:10161000300E8227A9EC0AF033C182F40401300EA7
:101620008227A9EC0AF06FEF14F00401760E826FA6
:10163000A9EC0AF00401310E826FA9EC0AF0040152
:101640002C0E826FA9EC0AF0AFEC23F0AFEC23F084
:101650001BEC23F002C600F103C601F101AF36EF27
:101660000BF00101FF0E026FFF0E036FBEEC22F0C4
:1016700029673DEF0BF042EF0BF004012D0E826F56
:10168000A9EC0AF02FC182F40401300E8227A9ECE4
:101690000AF030C182F40401300E8227A9EC0AF06E
:1016A00031C182F40401300E8227A9EC0AF032C164
:1016B00082F40401300E8227A9EC0AF033C182F4CF
:1016C0000401300E8227A9EC0AF004012C0E826F6F
:1016D000A9EC0AF01BEC23F004C600F105C601F1E9
:1016E00001AF78EF0BF00101FF0E026FFF0E036FE9
:1016F000BEEC22F029677FEF0BF084EF0BF00401C2
:101700002D0E826FA9EC0AF02FC182F40401300E75
:101710008227A9EC0AF030C182F40401300E82273E
:10172000A9EC0AF031C182F40401300E8227A9EC41
:101730000AF032C182F40401300E8227A9EC0AF0CB
:1017400033C182F40401300E8227A9EC0AF00401AF
:101750002C0E826FA9EC0AF01BEC23F006C600F1F8
:1017600007C601F101AFBAEF0BF00101FF0E026FE6
:10177000FF0E036FBEEC22F02967C1EF0BF0C6EF3E
:101780000BF004012D0E826FA9EC0AF02FC182F438
:101790000401300E8227A9EC0AF030C182F4040162
:1017A000300E8227A9EC0AF031C182F40401300E18
:1017B0008227A9EC0AF032C182F40401300E82279C
:1017C000A9EC0AF033C182F40401300E8227A9EC9F
:1017D0000AF06FEF14F00401760E826FA9EC0AF0A4
:1017E0000401320E826FA9EC0AF004012C0E826F04
:1017F000A9EC0AF017EC24F017EC24F01BEC23F012
:1018000008C600F109C601F101AF0CEF0CF00101AF
:10181000FF0E026FFF0E036FBEEC22F0296713EF7D
:101820000CF018EF0CF004012D0E826FA9EC0AF0F9
:101830002FC182F40401300E8227A9EC0AF030C1D6
:1018400082F40401300E8227A9EC0AF031C182F43F
:101850000401300E8227A9EC0AF032C182F404019F
:10186000300E8227A9EC0AF033C182F40401300E55
:101870008227A9EC0AF004012C0E826FA9EC0AF071
:101880001BEC23F00AC600F10BC601F101AF4EEFCD
:101890000CF00101FF0E026FFF0E036FBEEC22F091
:1018A000296755EF0CF05AEF0CF004012D0E826FF2
:1018B000A9EC0AF02FC182F40401300E8227A9ECB2
:1018C0000AF030C182F40401300E8227A9EC0AF03C
:1018D00031C182F40401300E8227A9EC0AF032C132
:1018E00082F40401300E8227A9EC0AF033C182F49D
:1018F0000401300E8227A9EC0AF004012C0E826F3D
:10190000A9EC0AF01BEC23F00CC600F10DC601F1A6
:1019100001AF90EF0CF00101FF0E026FFF0E036F9D
:10192000BEEC22F0296797EF0CF09CEF0CF004015D
:101930002D0E826FA9EC0AF02FC182F40401300E43
:101940008227A9EC0AF030C182F40401300E82270C
:10195000A9EC0AF031C182F40401300E8227A9EC0F
:101960000AF032C182F40401300E8227A9EC0AF099
:1019700033C182F40401300E8227A9EC0AF06FEF24
:1019800014F00401760E826FA9EC0AF00401330E04
:10199000826FA9EC0AF004012C0E826FA9EC0AF008
:1019A00085C382F4A9EC0AF0640E0D6E0301855123
:1019B000320A02E16A0E0D6E03018551330A02E11B
:1019C000700E0D6E03018551340A02E1760E0D6E24
:1019D00003018551350A02E17C0E0D6E030185512C
:1019E000360A02E1820E0D6E03018651780A65E027
:1019F0000DC00CF05CEC23F02981030187512D0A06
:101A0000D8B405EF0DF00101299188C32FF189C3E6
:101A100030F18AC331F18BC332F18CC333F169ECFD
:101A200023F0E0EC22F000C10BF09CEC07F001C1C8
:101A30000BF09CEC07F05CEC23F0298103018E5144
:101A40002D0AD8B426EF0DF0010129918FC32FF193
:101A500090C330F191C331F192C332F193C333F1AA
:101A600069EC23F0E0EC22F000C10BF09CEC07F0F5
:101A700001C10BF09CEC07F05CEC23F02981030121
:101A800095512D0AD8B447EF0DF00101299196C365
:101A90002FF197C330F198C331F199C332F19AC352
:101AA00033F169EC23F0E0EC22F000C10BF09CEC88
:101AB00007F001C10BF09CEC07F00DC00CF0BAEC84
:101AC00007F0BAEC07F0BAEC07F06FEF14F004017E
:101AD000760E826FA9EC0AF00401340E826FA9EC35
:101AE0000AF003018451780AD8B43FEF0EF03E0E9D
:101AF0000C6E5CEC23F02981030185512D0AD8B4CA
:101B000084EF0DF00101299186C32FF187C330F1D5
:101B100088C331F189C332F18AC333F169EC23F010
:101B2000E0EC22F000C10BF09CEC07F001C10BF0DF
:101B30009CEC07F05CEC23F0298103018C512D0A09
:101B4000D8B4A5EF0DF0010129918DC32FF18EC3FB
:101B500030F18FC331F190C332F191C333F169ECAD
:101B600023F0E0EC22F000C10BF09CEC07F001C187
:101B70000BF09CEC07F05CEC23F0298103019351FE
:101B80002D0AD8B4C6EF0DF00101299194C32FF1AD
:101B900095C330F196C331F197C332F198C333F155
:101BA00069EC23F0E0EC22F000C10BF09CEC07F0B4
:101BB00001C10BF09CEC07F05CEC23F029810301E0
:101BC0009A512D0AD8B4E7EF0DF0010129919BC37A
:101BD0002FF19CC330F19DC331F19EC332F19FC3FD
:101BE00033F169EC23F0E0EC22F000C10BF09CEC47
:101BF00007F001C10BF09CEC07F05CEC23F02981AD
:101C00000301A1512D0AD8B408EF0EF0010129916A
:101C1000A2C32FF1A3C330F1A4C331F1A5C332F1A4
:101C2000A6C333F169EC23F0E0EC22F000C10BF025
:101C30009CEC07F001C10BF09CEC07F05CEC23F08E
:101C400029810301A8512D0AD8B429EF0EF0010112
:101C50002991A9C32FF1AAC330F1ABC331F1ACC3B1
:101C600032F1ADC333F169EC23F0E0EC22F000C1B6
:101C70000BF09CEC07F001C10BF09CEC07F03E0E62
:101C80000C6EBAEC07F0BAEC07F0BAEC07F0BAEC5D
:101C900007F0BAEC07F0BAEC07F06FEF14F00301AD
:101CA0008351300AD8B410EF11F003018351310A87
:101CB000D8B41CEF12F003018351320AD8B488EF74
:101CC00012F003018351330AD8B496EF12F00301E6
:101CD0008351340AD8B4A4EF12F003018351350ABA
:101CE000D8B413EF14F003018351360AD8B441EF8E
:101CF00014F003018351460AD8B467EF13F00301CF
:101D000083514D0AD8B489EF0FF0030183516D0A56
:101D1000D8B4A3EF0FF0030183515A0AD8B496EF59
:101D200011F003018351490AD8B441EF15F00301C2
:101D30008351500AD8B473EF14F003018351540A4D
:101D4000D8B4ECEF14F003018351630AD8B4C3EFA5
:101D50000FF003018351430AD8B4BBEF10F0030125
:101D60008351730AD8B4C1EF0FF003018351610AA4
:101D7000D8B4D6EF0EF003018351650AD8B45EEFF4
:101D800011F003018351450AD8B46CEF11F003013F
:101D90008351620AD8B47AEF11F003018351420AE9
:101DA000D8B488EF11F0D8A45AEF1CF004014C0EFF
:101DB000826FA9EC0AF00401610E826FA9EC0AF0AF
:101DC00084EC25F004012C0E826FA9EC0AF01BECC8
:101DD00023F0ABC500F10101BEEC22F031C182F469
:101DE0000401300E8227A9EC0AF032C182F404010A
:101DF000300E8227A9EC0AF033C182F40401300EC0
:101E00008227A9EC0AF004012C0E826FA9EC0AF0DB
:101E10001BEC23F0ACC500F10101BEEC22F031C196
:101E200082F40401300E8227A9EC0AF032C182F458
:101E30000401300E8227A9EC0AF033C182F40401B8
:101E4000300E8227A9EC0AF004012C0E826FA9EC57
:101E50000AF01BEC23F0ADC500F10101BEEC22F04D
:101E600031C182F40401300E8227A9EC0AF032C19C
:101E700082F40401300E8227A9EC0AF033C182F407
:101E80000401300E8227A9EC0AF004012C0E826FA7
:101E9000A9EC0AF01BEC23F0AEC500F10101BEEC89
:101EA00022F031C182F40401300E8227A9EC0AF03D
:101EB00032C182F40401300E8227A9EC0AF033C14A
:101EC00082F40401300E8227A9EC0AF004012C0EE2
:101ED000826FA9EC0AF01BEC23F0B3C500F10101FD
:101EE000BEEC22F031C182F40401300E8227A9EC4D
:101EF0000AF032C182F40401300E8227A9EC0AF004
:101F000033C182F40401300E8227A9EC0AF06FEF8E
:101F100014F05CEC23F084C333F169EC23F0E0ECC3
:101F200022F0200E0C6E00C10BF09CEC07F000C1FB
:101F30002FF505012F51000A06E005012F51010A76
:101F400002E02AEC26F004014C0E826FA9EC0AF0A4
:101F500004014D0E826FA9EC0AF004012C0E826F71
:101F6000A9EC0AF01BEC23F02FC500F1BEEC22F027
:101F700033C182F40401300E8227A9EC0AF06FEF1E
:101F800014F04AEF2BF004014C0E826FA9EC0AF01A
:101F90000401630E826FA9EC0AF0D4EC24F0040172
:101FA0002C0E826FA9EC0AF0D8EC0FF06FEF14F052
:101FB0001BEC23F0B1C500F10101003B0F0E00172F
:101FC000BEEC22F033C182F40401300E8227A9EC6A
:101FD0000AF0B1C500F101010F0E01010017BEECBE
:101FE00022F033C182F40401300E8227A9EC0AF0FA
:101FF00004012D0E826FA9EC0AF0B0C500F10101B9
:10200000003B0F0E0017BEEC22F033C182F4040136
:10201000300E8227A9EC0AF0B0C500F101010F0EC5
:1020200001010017BEEC22F033C182F40401300E2E
:102030008227A9EC0AF004012D0E826FA9EC0AF0A8
:10204000AFC500F10101003B0F0E0017BEEC22F0FE
:1020500033C182F40401300E8227A9EC0AF0AFC527
:1020600000F101010F0E01010017BEEC22F033C197
:1020700082F40401300E8227A9EC0AF00401200E3C
:10208000826FA9EC0AF0AEC500F10F0E0101001736
:10209000BEEC22F033C182F40401300E8227A9EC99
:1020A0000AF00401200E826FA9EC0AF0ADC500F120
:1020B00001010101003B0F0E0017BEEC22F033C1FD
:1020C00082F40401300E8227A9EC0AF0ADC500F1BC
:1020D00001010F0E01010017BEEC22F033C182F4A2
:1020E0000401300E8227A9EC0AF004013A0E826F37
:1020F000A9EC0AF0ACC500F10101003B0F0E00177E
:10210000BEEC22F033C182F40401300E8227A9EC28
:102110000AF0ACC500F101010F0E01010017BEEC81
:1021200022F033C182F40401300E8227A9EC0AF0B8
:1021300004013A0E826FA9EC0AF0ABC500F101016F
:10214000003B0F0E0017BEEC22F033C182F40401F5
:10215000300E8227A9EC0AF0ABC500F101010F0E89
:102160000017BEEC22F033C182F40401300E822746
:10217000A9EC0AF0120084C3E8FF0F0BE83AE8CF9D
:10218000B1F585C3E8FF0F0B0501B11387C3E8FF65
:102190000F0BE83AE8CFB0F588C3E8FF0F0B050155
:1021A000B0138AC3E8FF0F0BE83AE8CFAFF58BC353
:1021B000E8FF0F0B0501AF138DC3E8FF0F0BE8CF4E
:1021C000AEF58FC3E8FF0F0BE83AE8CFADF590C34B
:1021D000E8FF0F0B0501AD1392C3E8FF0F0BE83AC0
:1021E000E8CFACF593C3E8FF0F0B0501AC1395C323
:1021F000E8FF0F0BE83AE8CFABF596C3E8FF0F0B0B
:102200000501AB1333EC25F004014C0E826FA9ECF1
:102210000AF00401430E826FA9EC0AF0CDEF0FF033
:102220000BEC2BF01BEC23F02DC500F1BEEC22F0E3
:1022300004014C0E826FA9EC0AF00401300E826F8B
:10224000A9EC0AF004012C0E826FA9EC0AF031C14E
:1022500082F40401300E8227A9EC0AF032C182F424
:102260000401300E8227A9EC0AF033C182F4040184
:10227000300E8227A9EC0AF004012C0E826FA9EC23
:102280000AF01BEC23F02EC500F1BEEC22F031C1A8
:1022900082F40401300E8227A9EC0AF032C182F4E4
:1022A0000401300E8227A9EC0AF033C182F4040144
:1022B000300E8227A9EC0AF06FEF14F004014C0EE7
:1022C000826FA9EC0AF00401650E826FA9EC0AF096
:1022D00013EC27F06FEF14F004014C0E826FA9ECA1
:1022E0000AF00401450E826FA9EC0AF030EC27F0E9
:1022F0006FEF14F004014C0E826FA9EC0AF0040198
:10230000620E826FA9EC0AF06AEC27F06FEF14F00E
:1023100004014C0E826FA9EC0AF00401420E826F98
:10232000A9EC0AF04DEC27F06FEF14F004014C0E0D
:10233000826FA9EC0AF004015A0E826FA9EC0AF030
:1023400004012C0E826FA9EC0AF00BEC2BF01BECB5
:1023500023F005012E51130A06E005012E51170A3C
:102360000DE0C7EF11F00101000E006F000E016FCC
:10237000100E026F000E036FC7EF11F00101000E87
:10238000006F000E016F000E026F010E036F01015E
:10239000100E046F000E056F000E066F000E076F23
:1023A00051EC22F0BEEC22F02AC182F40401300E7E
:1023B0008227A9EC0AF02BC182F40401300E822797
:1023C000A9EC0AF02CC182F40401300E8227A9EC9A
:1023D0000AF02DC182F40401300E8227A9EC0AF024
:1023E0002EC182F40401300E8227A9EC0AF02FC11D
:1023F00082F40401300E8227A9EC0AF030C182F485
:102400000401300E8227A9EC0AF031C182F40401E4
:10241000300E8227A9EC0AF032C182F40401300E9A
:102420008227A9EC0AF033C182F40401300E82271E
:10243000A9EC0AF06FEF14F004014C0E826FA9ECC6
:102440000AF00401310E826FA9EC0AF004012C0E8F
:10245000826FA9EC0AF025C500F126C501F127C558
:1024600002F128C503F10101100E046F000E056F83
:10247000000E066F000E076F51EC22F0BEEC22F04A
:102480002AC182F40401300E8227A9EC0AF02BC184
:1024900082F40401300E8227A9EC0AF02CC182F4E8
:1024A0000401300E8227A9EC0AF02DC182F4040148
:1024B000300E8227A9EC0AF02EC182F40401300EFE
:1024C0008227A9EC0AF02FC182F40401300E822782
:1024D000A9EC0AF030C182F40401300E8227A9EC85
:1024E0000AF031C182F40401300E8227A9EC0AF00F
:1024F00032C182F40401300E8227A9EC0AF033C104
:1025000082F40401300E8227A9EC0AF06FEF14F078
:1025100004014C0E826FA9EC0AF00401320E826FA6
:10252000A9EC0AF061EC29F06FEF14F004014C0EF5
:10253000826FA9EC0AF00401330E826FA9EC0AF055
:10254000BEEC29F026EF12F004014C0E826FA9ECCC
:102550000AF00401340E826FA9EC0AF004012C0E7B
:10256000826FA9EC0AF05CEC23F084C32AF185C3E6
:102570002BF186C32CF187C32DF188C32EF189C3BB
:102580002FF18AC330F18BC331F18CC332F18DC38B
:1025900033F10101296B69EC23F0E0EC22F0100E1D
:1025A000046F000E056F000E066F000E076F31EC12
:1025B00022F000C121F501C122F502C123F503C1BA
:1025C00024F5BEEC2AF034C5ABF535C5ACF536C5FF
:1025D000ADF537C5AEF538C5AFF539C5B0F53AC577
:1025E000B1F5D8EC0FF004012C0E826FA9EC0AF0C3
:1025F0003BC500F13CC501F13DC502F13EC503F10B
:102600000101000E046F000E056F010E066F000E33
:10261000076F51EC22F0BEEC22F0296712EF13F0A5
:1026200017EF13F004012D0E826FA9EC0AF030C1F0
:1026300082F40401300E8227A9EC0AF031C182F441
:102640000401300E8227A9EC0AF004012E0E826FDD
:10265000A9EC0AF032C182F40401300E8227A9EC01
:102660000AF033C182F40401300E8227A9EC0AF08B
:1026700004012C0E826FA9EC0AF01BEC23F03FC57D
:1026800000F140C501F184EC1DF004012C0E826FB5
:10269000A9EC0AF01BEC23F041C500F1BEEC22F0DE
:1026A00031C182F40401300E8227A9EC0AF032C154
:1026B00082F40401300E8227A9EC0AF033C182F4BF
:1026C0000401300E8227A9EC0AF06FEF14F05CECE5
:1026D00023F085C32AF186C32BF187C32CF188C36D
:1026E0002DF189C32EF18AC32FF18BC330F18CC336
:1026F00031F18DC332F18EC333F10101296B69ECE5
:1027000023F0E0EC22F00101010E046F000E056FD2
:10271000000E066F000E076F20EC22F0100E046F03
:10272000000E056F000E066F000E076F31EC22F0F1
:1027300000C129F501C12AF502C12BF503C12CF511
:10274000EAEC28F004014C0E826FA9EC0AF00401B7
:10275000460E826FA9EC0AF004012C0E826FA9ECE0
:102760000AF025C500F126C501F127C502F128C5EB
:1027700003F10101100E046F000E056F000E066FCD
:10278000000E076F51EC22F0BEEC22F02AC182F459
:102790000401300E8227A9EC0AF02BC182F4040157
:1027A000300E8227A9EC0AF02CC182F40401300E0D
:1027B0008227A9EC0AF02DC182F40401300E822791
:1027C000A9EC0AF02EC182F40401300E8227A9EC94
:1027D0000AF02FC182F40401300E8227A9EC0AF01E
:1027E00030C182F40401300E8227A9EC0AF031C115
:1027F00082F40401300E8227A9EC0AF032C182F47F
:102800000401300E8227A9EC0AF033C182F40401DE
:10281000300E8227A9EC0AF06FEF14F00F98BEEC8F
:1028200029F06FEF14F004014C0E826FA9EC0AF04E
:102830000401350E826FA9EC0AF004012C0E826FA0
:10284000A9EC0AF01BEC23F00784B5C500F107944E
:10285000BEEC22F031C182F40401300E8227A9ECD3
:102860000AF032C182F40401300E8227A9EC0AF08A
:1028700033C182F40401300E8227A9EC0AF06FEF15
:1028800014F081EC29F01BEC23F033C500F1BEEC11
:1028900022F004014C0E826FA9EC0AF00401360EFE
:1028A000826FA9EC0AF004012C0E826FA9EC0AF0E9
:1028B00031C182F40401300E8227A9EC0AF032C142
:1028C00082F40401300E8227A9EC0AF033C182F4AD
:1028D0000401300E8227A9EC0AF06FEF14F0B3EC7C
:1028E0000AF05AEF1CF004014C0E826FA9EC0AF0BA
:1028F0000401500E826FA9EC0AF004012C0E826FC5
:10290000A9EC0AF085C32AF186C32BF187C32CF109
:1029100088C32DF189C32EF18AC32FF18BC330F107
:102920008CC331F18DC332F18EC333F1010169ECF7
:1029300023F0E0EC22F003018451530A0DE003017F
:1029400084514D0A38E00401780E826FA9EC0AF038
:10295000B3EC0AF05AEF1CF00401530E826FA9EC9D
:102960000AF0250E0C6E00C10BF09CEC07F0260E51
:102970000C6E01C10BF09CEC07F0270E0C6E02C12F
:102980000BF09CEC07F0280E0C6E03C10BF09CECD6
:1029900007F000C153F501C154F502C155F503C15B
:1029A00056F500C157F501C158F502C159F503C1EB
:1029B0005AF550EF15F004014D0E826FA9EC0AF0A4
:1029C000290E0C6E00C10BF09CEC07F000C15BF50A
:1029D00000C15CF550EF15F004014C0E826FA9ECBC
:1029E0000AF00401540E826FA9EC0AF004012C0EC7
:1029F000826FA9EC0AF084C32AF185C32BF186C348
:102A00002CF187C32DF188C32EF189C32FF18AC31E
:102A100030F18BC331F18DC332F18EC333F101013B
:102A200069EC23F0E0EC22F00101000E046F000ECF
:102A3000056F010E066F000E076F31EC22F0210EBC
:102A40000C6E00C10BF09CEC07F0220E0C6E01C165
:102A50000BF09CEC07F0230E0C6E02C10BF09CEC0B
:102A600007F0240E0C6E03C10BF09CEC07F000C1C4
:102A70005DF501C15EF502C15FF503C160F550EF80
:102A800015F004014C0E826FA9EC0AF00401490E06
:102A9000826FA9EC0AF004012C0E826FA9EC0AF0F7
:102AA000250EB3EC07F0E8CF00F1260EB3EC07F0EB
:102AB000E8CF01F1270EB3EC07F0E8CF02F1280EC2
:102AC000B3EC07F0E8CF03F1BEEC22F0A1EC20F06C
:102AD0000401730E826FA9EC0AF004012C0E826FC0
:102AE000A9EC0AF01BEC23F0290EB3EC07F0E8CFB9
:102AF00000F1BEEC22F0A1EC20F00401730E826F15
:102B0000A9EC0AF004012C0E826FA9EC0AF057C55B
:102B100000F158C501F159C502F15AC503F1BEECE7
:102B200022F0A1EC20F00401730E826FA9EC0AF0F0
:102B300004012C0E826FA9EC0AF01BEC23F05CC59B
:102B400000F1BEEC22F0A1EC20F004016D0E826FCA
:102B5000A9EC0AF004012C0E826FA9EC0AF05DC505
:102B600000F15EC501F15FC502F160C503F175ECCE
:102B70001CF004012C0E826FA9EC0AF0B3EC0AF0F1
:102B80005AEF1CF083C32AF184C32BF185C32CF1C7
:102B900086C32DF187C32EF188C32FF189C330F18D
:102BA0008AC331F18BC332F18CC333F1010169EC7B
:102BB00023F0E0EC22F0160E0C6E00C10BF09CEC42
:102BC00007F0170E0C6E01C10BF09CEC07F0180E0D
:102BD0000C6E02C10BF09CEC07F0190E0C6E03C1D9
:102BE0000BF09CEC07F000C18AF101C18BF102C12E
:102BF0008CF103C18DF100C18EF101C18FF102C1D1
:102C000090F103C191F1A4EF16F083C32AF184C3BC
:102C10002BF185C32CF186C32DF187C32EF188C318
:102C20002FF189C330F18AC331F18BC332F18CC3E8
:102C300033F1010169EC23F0E0EC22F000C18AF1EC
:102C400001C18BF102C18CF103C18DF100C18EF184
:102C500001C18FF102C190F103C191F1A4EF16F00F
:102C600083C32AF184C32BF185C32CF186C32DF1D4
:102C700087C32EF188C32FF189C330F18AC331F1A4
:102C80008CC332F18DC333F1010169EC23F0E0EC28
:102C900022F00101000E046F000E056F010E066F99
:102CA000000E076F31EC22F01A0E0C6E00C10BF013
:102CB0009CEC07F01B0E0C6E01C10BF09CEC07F0B6
:102CC0001C0E0C6E02C10BF09CEC07F01D0E0C6E7E
:102CD00003C10BF09CEC07F000C192F101C193F12C
:102CE00002C194F103C195F1A4EF16F083C32AF158
:102CF00084C32BF185C32CF186C32DF187C32EF13C
:102D000088C32FF189C330F18AC331F18CC332F10A
:102D10008DC333F1010169EC23F0E0EC22F00101F5
:102D2000000E046F000E056F010E066F000E076F98
:102D300031EC22F000C192F101C193F102C194F192
:102D400003C195F1A4EF16F0160EB3EC07F0E8CF2F
:102D500000F1170EB3EC07F0E8CF01F1180EB3EC59
:102D600007F0E8CF02F1190EB3EC07F0E8CF03F15A
:102D7000BEEC22F0A1EC20F00401730E826FA9ECEE
:102D80000AF004012C0E826FA9EC0AF08AC100F14E
:102D90008BC101F18CC102F18DC103F1BEEC22F0B7
:102DA000A1EC20F00401730E826FA9EC0AF004017B
:102DB0002C0E826FA9EC0AF01A0EB3EC07F0E8CFE4
:102DC00000F11B0EB3EC07F0E8CF01F11C0EB3ECE1
:102DD00007F0E8CF02F11D0EB3EC07F0E8CF03F1E6
:102DE00075EC1CF004012C0E826FA9EC0AF092C164
:102DF00000F193C101F194C102F195C103F175ECA9
:102E00001CF0B3EC0AF05AEF1CF00401690E826F5B
:102E1000A9EC0AF004012C0E826FA9EC0AF0010162
:102E2000040E006F000E016F000E026F000E036FA4
:102E3000BEEC22F02CC182F40401300E8227A9ECF2
:102E40000AF02DC182F40401300E8227A9EC0AF0A9
:102E50002EC182F40401300E8227A9EC0AF02FC1A2
:102E600082F40401300E8227A9EC0AF030C182F40A
:102E70000401300E8227A9EC0AF031C182F404016A
:102E8000300E8227A9EC0AF032C182F40401300E20
:102E90008227A9EC0AF033C182F40401300E8227A4
:102EA000A9EC0AF004012C0E826FA9EC0AF00101D2
:102EB0000B0E006F000E016F000E026F000E036F0D
:102EC000BEEC22F02CC182F40401300E8227A9EC62
:102ED0000AF02DC182F40401300E8227A9EC0AF019
:102EE0002EC182F40401300E8227A9EC0AF02FC112
:102EF00082F40401300E8227A9EC0AF030C182F47A
:102F00000401300E8227A9EC0AF031C182F40401D9
:102F1000300E8227A9EC0AF032C182F40401300E8F
:102F20008227A9EC0AF033C182F40401300E822713
:102F3000A9EC0AF004012C0E826FA9EC0AF0010141
:102F40001B0E006F000E016F000E026F000E036F6C
:102F5000BEEC22F02CC182F40401300E8227A9ECD1
:102F60000AF02DC182F40401300E8227A9EC0AF088
:102F70002EC182F40401300E8227A9EC0AF02FC181
:102F800082F40401300E8227A9EC0AF030C182F4E9
:102F90000401300E8227A9EC0AF031C182F4040149
:102FA000300E8227A9EC0AF032C182F40401300EFF
:102FB0008227A9EC0AF033C182F40401300E822783
:102FC000A9EC0AF004012C0E826FA9EC0AF0200E85
:102FD000F86EF76AF66A04010900F5CF82F4A9ECED
:102FE0000AF00900F5CF82F4A9EC0AF00900F5CF48
:102FF00082F4A9EC0AF00900F5CF82F4A9EC0AF0FA
:103000000900F5CF82F4A9EC0AF00900F5CF82F4AB
:10301000A9EC0AF00900F5CF82F4A9EC0AF0090046
:10302000F5CF82F4A9EC0AF0B3EC0AF05AEF1CF0E9
:103030008351630AD8A45AEF1CF08451610AD8A4C2
:103040005AEF1CF085516C0AD8A45AEF1CF0865137
:10305000410A42E08651440A1BE08651420AD8B434
:103060007FEF18F08651350AD8B4E4EF1DF0865191
:10307000360AD8B439EF1EF08651370AD8B4A2EF19
:103080001EF08651380AD8B400EF1FF05AEF1CF03A
:103090000798079A04017A0E826FA9EC0AF00401DE
:1030A000780E826FA9EC0AF00401640E826FA9EC1D
:1030B0000AF081A863EF18F00401550E826FA9ECA5
:1030C0000AF068EF18F004014C0E826FA9EC0AF0C8
:1030D000B3EC0AF05AEF1CF00788079A04017A0E45
:1030E000826FA9EC0AF00401410E826FA9EC0AF08C
:1030F0000401610E826FA9EC0AF059EF18F00798ED
:10310000078A04017A0E826FA9EC0AF00401420ECC
:10311000826FA9EC0AF00401610E826FA9EC0AF03B
:1031200059EF18F0010166679DEF18F067679DEF92
:1031300018F068679DEF18F06967B5EF18F04F67F2
:10314000A9EF18F05067A9EF18F05167A9EF18F030
:103150005267B5EF18F00101000E006F000E016F0D
:10316000000E026F000E036F12000101620E046F69
:10317000010E056F000E066F000E076F66C100F1AD
:1031800067C101F168C102F169C103F120EC22F0CD
:1031900003BF39EF19F00101000E046FA80E056F8F
:1031A000550E066F020E076F66C100F167C101F18F
:1031B00068C102F169C103F166C186F167C187F197
:1031C00068C188F169C189F120EC22F003BFF2EFF8
:1031D00018F00101000E866FA80E876F550E886FDC
:1031E000020E896F0E0EB3EC07F0E8CF18F10F0E48
:1031F000B3EC07F0E8CF19F1100EB3EC07F0E8CF0D
:103200001AF1110EB3EC07F0E8CF1BF169EC21F0D5
:1032100086C104F187C105F188C106F189C107F1B2
:1032200020EC22F007822DEC21F069EC21F00792CE
:103230002DEC21F086C100F187C101F188C102F1B6
:1032400089C103F107922DEC21F0CC0E046FE00E42
:10325000056F870E066F050E076F20EC22F000C188
:1032600018F101C119F102C11AF103C11BF171EF8B
:1032700019F00101800E006F1A0E016F060E026F29
:10328000000E036F4FC104F150C105F151C106F1A9
:1032900052C107F120EC22F003AF52EF19F01BEC02
:1032A00023F012000E0EB3EC07F0E8CF18F10F0E6A
:1032B000B3EC07F0E8CF19F1100EB3EC07F0E8CF4C
:1032C0001AF1110EB3EC07F0E8CF1BF14FC100F17A
:1032D00050C101F151C102F152C103F107822DEC3D
:1032E00021F018C100F119C101F11AC102F11BC18D
:1032F00003F112000401730E826FA9EC0AF00401BD
:103300002C0E826FA9EC0AF0078462C166F163C1DA
:1033100067F164C168F165C169F14BC14FF14CC1FE
:1033200050F14DC151F14EC152F157C159F158C13F
:103330005AF10794A0EC19F0B3EC0AF05AEF1CF024
:1033400066C100F167C101F168C102F169C103F111
:103350000101BEEC22F0A1EC20F00401630E826FAB
:10336000A9EC0AF004012C0E826FA9EC0AF04FC1FF
:1033700000F150C101F151C102F152C103F101014B
:10338000BEEC22F0A1EC20F00401660E826FA9ECE5
:103390000AF004012C0E826FA9EC0AF01BEC23F05A
:1033A00059C100F15AC101F10101BEEC22F0A1ECBA
:1033B00020F00401740E826FA9EC0AF01200108252
:1033C0000401530E826FA9EC0AF004012C0E826FE7
:1033D000A9EC0AF083C32AF184C32BF185C32CF135
:1033E00086C32DF187C32EF188C32FF189C330F135
:1033F0008AC331F18BC332F18CC333F1010169EC23
:1034000023F0E0EC22F000C166F101C167F102C1D6
:1034100068F103C169F18EC32AF18FC32BF190C308
:103420002CF191C32DF192C32EF193C32FF194C3CC
:1034300030F195C331F196C332F197C333F10101F5
:1034400069EC23F0E0EC22F000C14FF101C150F132
:1034500002C151F103C152F15CEC23F099C32FF189
:103460009AC330F19BC331F19CC332F19DC333F158
:10347000010169EC23F0E0EC22F000C159F101C137
:103480005AF1A0EC19F004012C0E826FA9EC0AF09D
:1034900051EF1AF08251520A03E10F8251EF1AF0F4
:1034A0000F928251750A03E1108458EF1AF01094BC
:1034B0008251550A03E110865FEF1AF010960784D7
:1034C00010B2BCEF1AF010A4A8EF1AF0B6C166F162
:1034D000B7C167F1B8C168F1B9C169F1BAC16AF1A0
:1034E000BBC16BF1BCC16CF1BDC16DF1BEC16EF170
:1034F000BFC16FF1C0C170F1C1C171F1C2C172F140
:10350000C3C173F1C4C174F1C5C175F1C6C176F10F
:10351000C7C177F1C8C178F1C9C179F1CAC17AF1DF
:10352000CBC17BF1CCC17CF1CDC17DF1CEC17EF1AF
:10353000CFC17FF1D0C180F1D1C181F1D2C182F17F
:10354000D3C183F1D4C184F1D5C185F1B0EF1AF0B4
:1035500062C166F163C167F164C168F165C169F177
:103560004BC14FF14CC150F14DC151F14EC152F11F
:1035700057C159F158C15AF107940FA0DEEF1AF064
:1035800001019267CBEF1AF09367CBEF1AF09467C3
:10359000CBEF1AF09567CFEF1AF0DEEF1AF092EC4E
:1035A00018F092C104F193C105F194C106F195C1DF
:1035B00007F120EC22F003BF22EF1CF092EC18F090
:1035C0000101000E046F000E056F010E066F000E64
:1035D000076F51EC22F010A4F5EF1AF00401750EFC
:1035E000826FA9EC0AF0FAEF1AF00401720E826FF2
:1035F000A9EC0AF004012C0E826FA9EC0AF0BEECD3
:1036000022F0296709EF1BF00401200E826F0CEFF6
:103610001BF004012D0E826FA9EC0AF030C182F478
:103620000401300E8227A9EC0AF031C182F40401B2
:10363000300E8227A9EC0AF004012E0E826FA9EC4D
:103640000AF032C182F40401300E8227A9EC0AF09C
:1036500033C182F40401300E8227A9EC0AF0040180
:103660006D0E826FA9EC0AF004012C0E826FA9EC9A
:103670000AF04FC100F150C101F151C102F152C134
:1036800003F10101BEEC22F0A1EC20F00401480E90
:10369000826FA9EC0AF004017A0E826FA9EC0AF09D
:1036A00004012C0E826FA9EC0AF066C100F167C11B
:1036B00001F168C102F169C103F10101BEEC22F020
:1036C000A1EC20F00401630E826FA9EC0AF0040162
:1036D0002C0E826FA9EC0AF066C100F167C101F1FE
:1036E00068C102F169C103F101010A0E046F000E05
:1036F000056F000E066F000E076F31EC22F0000E12
:10370000046F120E056F000E066F000E076F51EC6E
:1037100022F0BEEC22F02AC182F40401300E82278E
:10372000A9EC0AF02BC182F40401300E8227A9EC27
:103730000AF02CC182F40401300E8227A9EC0AF0B1
:103740002DC182F40401300E8227A9EC0AF02EC1AB
:1037500082F40401300E8227A9EC0AF02FC182F412
:103760000401300E8227A9EC0AF030C182F4040172
:10377000300E8227A9EC0AF004012E0E826FA9EC0C
:103780000AF031C182F40401300E8227A9EC0AF05C
:1037900032C182F40401300E8227A9EC0AF033C151
:1037A00082F40401300E8227A9EC0AF00401730EA2
:1037B000826FA9EC0AF004012C0E826FA9EC0AF0CA
:1037C0001BEC23F059C100F15AC101F184EC1DF04A
:1037D0000FB2EEEF1BF00FA020EF1CF004012C0E37
:1037E000826FA9EC0AF0200EF86EF76AF66A0401FF
:1037F0000900F5CF82F4A9EC0AF00900F5CF82F4B4
:10380000A9EC0AF00900F5CF82F4A9EC0AF009004E
:10381000F5CF82F4A9EC0AF00900F5CF82F4A9EC07
:103820000AF00900F5CF82F4A9EC0AF00900F5CFFF
:1038300082F4A9EC0AF00900F5CF82F4A9EC0AF0B1
:10384000B3EC0AF00F905AEF1CF00401630E826F84
:10385000A9EC0AF004012C0E826FA9EC0AF060ECCE
:103860001CF004012C0E826FA9EC0AF0D3EC1CF0C2
:1038700004012C0E826FA9EC0AF04FEC1DF004013C
:103880002C0E826FA9EC0AF00101F80E006FCD0E2C
:10389000016F660E026F030E036F75EC1CF00401DE
:1038A0002C0E826FA9EC0AF065EC1DF0B3EC0AF067
:1038B0005AEF1CF00301C26B0790109269EF1FF0E2
:1038C000D8900E0EB3EC07F0E8CF00F10F0EB3EC7A
:1038D00007F0E8CF01F1100EB3EC07F0E8CF02F1EA
:1038E000110EB3EC07F0E8CF03F10101000E046FF5
:1038F000000E056F010E066F000E076F51EC22F0EF
:10390000BEEC22F02AC182F40401300E8227A9EC19
:103910000AF02BC182F40401300E8227A9EC0AF0D0
:103920002CC182F40401300E8227A9EC0AF02DC1CB
:1039300082F40401300E8227A9EC0AF02EC182F431
:103940000401300E8227A9EC0AF02FC182F4040191
:10395000300E8227A9EC0AF030C182F40401300E47
:103960008227A9EC0AF031C182F40401300E8227CB
:10397000A9EC0AF004012E0E826FA9EC0AF032C104
:1039800082F40401300E8227A9EC0AF033C182F4DC
:103990000401300E8227A9EC0AF004016D0E826F3B
:1039A000A9EC0AF01200120EB3EC07F0E8CF00F118
:1039B000130EB3EC07F0E8CF01F1140EB3EC07F0EF
:1039C000E8CF02F1150EB3EC07F0E8CF03F10101E7
:1039D0000A0E046F000E056F000E066F000E076FD3
:1039E00031EC22F0000E046F120E056F000E066F10
:1039F000000E076F51EC22F0BEEC22F02AC182F4D7
:103A00000401300E8227A9EC0AF02BC182F40401D4
:103A1000300E8227A9EC0AF02CC182F40401300E8A
:103A20008227A9EC0AF02DC182F40401300E82270E
:103A3000A9EC0AF02EC182F40401300E8227A9EC11
:103A40000AF02FC182F40401300E8227A9EC0AF09B
:103A500030C182F40401300E8227A9EC0AF004017F
:103A60002E0E826FA9EC0AF031C182F40401300EEF
:103A70008227A9EC0AF032C182F40401300E8227B9
:103A8000A9EC0AF033C182F40401300E8227A9ECBC
:103A90000AF00401730E826FA9EC0AF012000A0EFC
:103AA000B3EC07F0E8CF00F10B0EB3EC07F0E8CF72
:103AB00001F10C0EB3EC07F0E8CF02F10D0EB3EC00
:103AC00007F0E8CF03F184EF1DF0060EB3EC07F02A
:103AD000E8CF00F1070EB3EC07F0E8CF01F1080ED4
:103AE000B3EC07F0E8CF02F1090EB3EC07F0E8CF32
:103AF00003F184EF1DF001011BEC23F0078457C193
:103B000000F158C101F107940101E80E046F800E25
:103B1000056F000E066F000E076F31EC22F0000EED
:103B2000046F040E056F000E066F000E076F51EC58
:103B300022F0880E046F130E056F000E066F000E44
:103B4000076F20EC22F00A0E046F000E056F000EC6
:103B5000066F000E076F51EC22F0BEEC22F001015F
:103B60002967B8EF1DF00401200E826FBBEF1DF036
:103B700004012D0E826FA9EC0AF030C182F4040119
:103B8000300E8227A9EC0AF031C182F40401300E14
:103B90008227A9EC0AF032C182F40401300E822798
:103BA000A9EC0AF004012E0E826FA9EC0AF033C1D1
:103BB00082F40401300E8227A9EC0AF00401430EBE
:103BC000826FA9EC0AF0120087C32AF188C32BF197
:103BD00089C32CF18AC32DF18BC32EF18CC32FF135
:103BE0008DC330F18EC331F190C332F191C333F103
:103BF0000101296B69EC23F0E0EC22F00101000ED9
:103C0000046F000E056F010E066F000E076F31EC9A
:103C100022F00E0E0C6E00C10BF09CEC07F00F0EA4
:103C20000C6E01C10BF09CEC07F0100E0C6E02C183
:103C30000BF09CEC07F0110E0C6E03C10BF09CEC2A
:103C400007F004017A0E826FA9EC0AF004012C0E31
:103C5000826FA9EC0AF00401350E826FA9EC0AF01C
:103C600004012C0E826FA9EC0AF060EC1CF068EFE6
:103C700018F087C32AF188C32BF189C32CF18AC3BA
:103C80002DF18BC32EF18CC32FF18DC330F18EC378
:103C900031F190C332F191C333F10101296B69EC29
:103CA00023F0E0EC22F0880E046F130E056F000E77
:103CB000066F000E076F25EC22F0000E046F040E55
:103CC000056F000E066F000E076F31EC22F0010148
:103CD000E80E046F800E056F000E066F000E076F72
:103CE00051EC22F00A0E0C6E00C10BF09CEC07F0B8
:103CF0000B0E0C6E01C10BF09CEC07F00C0E0C6E61
:103D000002C10BF09CEC07F00D0E0C6E03C10BF022
:103D10009CEC07F004017A0E826FA9EC0AF0040112
:103D20002C0E826FA9EC0AF00401360E826FA9EC0A
:103D30000AF004012C0E826FA9EC0AF04FEC1DF082
:103D400068EF18F087C32AF188C32BF189C32CF1DF
:103D50008AC32DF18BC32EF18CC32FF18DC330F1AB
:103D60008FC331F190C332F191C333F1010169EC9A
:103D700023F0E0EC22F0000E046F120E056F000E2F
:103D8000066F000E076F31EC22F001010A0E046F7E
:103D9000000E056F000E066F000E076F51EC22F04B
:103DA000120E0C6E00C10BF09CEC07F0130E0C6EA3
:103DB00001C10BF09CEC07F0140E0C6E02C10BF06D
:103DC0009CEC07F0150E0C6E03C10BF09CEC07F099
:103DD00004017A0E826FA9EC0AF004012C0E826FA6
:103DE000A9EC0AF00401370E826FA9EC0AF0040175
:103DF0002C0E826FA9EC0AF0D3EC1CF068EF18F0DF
:103E000087C32AF188C32BF189C32CF18AC32DF112
:103E10008BC32EF18CC32FF18DC330F18EC331F1E2
:103E200090C332F191C333F10101296B69EC23F0A6
:103E3000E0EC22F0880E046F130E056F000E066F83
:103E4000000E076F25EC22F0000E046F040E056FC4
:103E5000000E066F000E076F31EC22F00101E80E34
:103E6000046F800E056F000E066F000E076F51EC99
:103E700022F0060E0C6E00C10BF09CEC07F0070E52
:103E80000C6E01C10BF09CEC07F0080E0C6E02C129
:103E90000BF09CEC07F0090E0C6E03C10BF09CECD0
:103EA00007F004017A0E826FA9EC0AF004012C0ECF
:103EB000826FA9EC0AF00401380E826FA9EC0AF0B7
:103EC00004012C0E826FA9EC0AF065EC1DF068EF7E
:103ED00018F081A827EF20F007A8E0EF1FF00101FC
:103EE000800E006F1A0E016F060E026F000E036F38
:103EF0004BC104F14CC105F14DC106F14EC107F1B2
:103F000020EC22F003BF27EF20F09BEC20F04BC108
:103F100000F14CC101F14DC102F14EC103F1078224
:103F20002DEC21F018C104F119C105F11AC106F1F7
:103F30001BC107F1F80E006FCD0E016F660E026F08
:103F4000030E036F20EC22F00E0E0C6E00C10BF07E
:103F50009CEC07F00F0E0C6E01C10BF09CEC07F00F
:103F6000100E0C6E02C10BF09CEC07F0110E0C6EE3
:103F700003C10BF09CEC07F0078401011BEC23F05C
:103F800057C100F158C101F107940A0E0C6E00C12F
:103F90000BF09CEC07F00B0E0C6E01C10BF09CECCF
:103FA00007F00C0E0C6E02C10BF09CEC07F00D0E2E
:103FB0000C6E03C10BF09CEC07F0079827EF20F084
:103FC00007AA27EF20F0078401011BEC23F057C15B
:103FD00000F158C101F10794060E0C6E00C10BF000
:103FE0009CEC07F0070E0C6E01C10BF09CEC07F087
:103FF000080E0C6E02C10BF09CEC07F0090E0C6E63
:1040000003C10BF09CEC07F0078462C100F163C1AF
:1040100001F164C102F165C103F10794120E0C6E47
:1040200000C10BF09CEC07F0130E0C6E01C10BF0FD
:104030009CEC07F0140E0C6E02C10BF09CEC07F028
:10404000150E0C6E03C10BF09CEC07F0079A0401EF
:10405000805181197F0B0BE09EA809D014EE00F06F
:1040600081517F0BE126E750812B0F01AD6E0501D9
:104070002F51010A13E081AA4EEF20F005012F51C4
:10408000000A0AE00FB84EEF20F0050130674EEF4E
:1040900020F00FB84EEF20F04AEF2BF081B863EF1D
:1040A00020F084EC25F005012F51020A02E063EFB5
:1040B00020F05C2F63EF20F05BC55CF50501010E7D
:1040C000306F3C0E316F12EF0AF018C100F119C1C8
:1040D00001F11AC102F11BC103F1000E046F000EC1
:1040E000056F010E066F000E076F51EC22F029A13B
:1040F00090EF20F02051D8B490EF20F018C100F1DB
:1041000019C101F11AC102F11BC103F1000E046FC4
:10411000000E056F0A0E066F000E076F51EC22F0BD
:10412000120001010451001305510113065102133D
:104130000751031312000101186B196B1A6B1B6BEB
:1041400012002AC182F40401300E8227A9EC0AF081
:104150002BC182F40401300E8227A9EC0AF02CC195
:1041600082F40401300E8227A9EC0AF02DC182F4FA
:104170000401300E8227A9EC0AF02EC182F404015A
:10418000300E8227A9EC0AF02FC182F40401300E10
:104190008227A9EC0AF030C182F40401300E822794
:1041A000A9EC0AF031C182F40401300E8227A9EC97
:1041B0000AF032C182F40401300E8227A9EC0AF021
:1041C00033C182F40401300E8227A9EC0AF01200F8
:1041D0002FC182F40401300E8227A9EC0AF030C10D
:1041E00082F40401300E8227A9EC0AF031C182F476
:1041F0000401300E8227A9EC0AF032C182F40401D6
:10420000300E8227A9EC0AF033C182F40401300E8B
:104210008227A9EC0AF01200060E116E060E126E2D
:10422000060E136E112E12EF21F0122E12EF21F056
:10423000132E12EF21F08B84020E116E020E126EFD
:10424000020E136E112E22EF21F0122E22EF21F01A
:10425000132E22EF21F08B9412000101005305E18F
:10426000015303E1025301E1002BF0EC21F01BECC0
:1042700023F03951006F3A51016F420E046F4B0E1B
:10428000056F000E066F000E076F31EC22F000C1C3
:1042900004F101C105F102C106F103C107F118C122
:1042A00000F119C101F11AC102F11BC103F107B2FA
:1042B0005EEF21F025EC22F060EF21F020EC22F0FF
:1042C00000C118F101C119F102C11AF103C11BF1BA
:1042D00012001BEC23F059C100F15AC101F1060E86
:1042E000B3EC07F0E8CF04F1070EB3EC07F0E8CF2A
:1042F00005F1080EB3EC07F0E8CF06F1090EB3ECB8
:1043000007F0E8CF07F120EC22F000C124F101C151
:1043100025F102C126F103C127F1290E046F000E19
:10432000056F000E066F000E076F31EC22F0EE0EE7
:10433000046F430E056F000E066F000E076F25EC2D
:1043400022F024C104F125C105F126C106F127C1DF
:1043500007F131EC22F000C11CF101C11DF102C1D5
:104360001EF103C11FF1120EB3EC07F0E8CF04F108
:10437000130EB3EC07F0E8CF05F1140EB3EC07F021
:10438000E8CF06F1150EB3EC07F0E8CF07F10D0EFC
:10439000006F000E016F000E026F000E036F31EC14
:1043A00022F0180E046F000E056F000E066F000E4F
:1043B000076F51EC22F01CC104F11DC105F11EC1B3
:1043C00006F11FC107F125EC22F06A0E046F2A0ED8
:1043D000056F000E066F000E076F20EC22F0120032
:1043E000BF0EFA6E200E3A6F396BD8900037013746
:1043F00002370337D8B001EF22F03A2FF6EF21F061
:1044000039073A070353D8B412000331070B800968
:104410003F6F03390F0B010F396F80EC5FF0406F76
:10442000390580EC5FF0405D405F396B3F33D8B0B9
:10443000392739333FA916EF22F0405139271200AE
:10444000010140EC23F0D8B012000101035107191B
:10445000346F03EC23F0D8900751031934AF800F69
:1044600012000101346B27EC23F0D8A03DEC23F0BF
:10447000D8B0120012EC23F01BEC23F01F0E366FA5
:1044800053EC23F00B35D8B003EC23F0D8A0033560
:10449000D8B01200362F40EF22F034B12AEC23F0CE
:1044A00012000101346B04510511061107110008B7
:1044B000D8A027EC23F0D8A03DEC23F0D8B0120010
:1044C000086B096B0A6B0B6B53EC23F01F0E366FF6
:1044D00053EC23F007510B5DD8A47BEF22F006517B
:1044E0000A5DD8A47BEF22F00551095DD8A47BEFCB
:1044F00022F00451085DD8A08EEF22F00451085F2D
:104500000551D8A0053D095F0651D8A0063D0A5FB8
:104510000751D8A0073D0B5FD8900081362F68EF78
:1045200022F034B12AEC23F0346B27EC23F0D8903E
:1045300057EC23F007510B5DD8A4ABEF22F00651E6
:104540000A5DD8A4ABEF22F00551095DD8A4ABEF0A
:1045500022F00451085DD8A0BAEF22F0003FBAEF74
:1045600022F0013FBAEF22F0023FBAEF22F0032B14
:10457000D8B4120034B12AEC23F012000101346BDC
:1045800027EC23F0D8B012005CEC23F0200E366F3D
:10459000003701370237033711EE33F00A0E376F59
:1045A000E7360A0EE75CD8B0E76EE552372FD0EF5A
:1045B00022F0362FC8EF22F034B12981D8901200B2
:1045C00001010A0E346F200E366F11EE29F03451BE
:1045D000376F0A0ED890E652D8B0E726E732372F69
:1045E000EBEF22F00333023301330033362FE5EFD4
:1045F00022F0E750FF0FD8A00335D8B0120029B140
:104600002AEC23F01200045100270551D8B0053DD3
:1046100001270651D8B0063D02270751D8B0073D03
:10462000032712000051086F0151096F02510A6FF0
:1046300003510B6F12000101006B016B026B036BE6
:1046400012000101046B056B066B076B120003354A
:10465000D8A012000351800B001F011F021F031F6F
:10466000003F3AEF23F0013F3AEF23F0023F3AEFE9
:1046700023F0032B342B032512000735D8A012009A
:104680000751800B041F051F061F071F043F50EF33
:1046900023F0053F50EF23F0063F50EF23F0072BA8
:1046A000342B07251200003701370237033708374C
:1046B00009370A370B3712000101296B2A6B2B6B64
:1046C0002C6B2D6B2E6B2F6B306B316B326B336B16
:1046D000120001012A510F0B2A6F2B510F0B2B6F68
:1046E0002C510F0B2C6F2D510F0B2D6F2E510F0BCB
:1046F0002E6F2F510F0B2F6F30510F0B306F315129
:104700000F0B316F32510F0B326F33510F0B336F71
:1047100012008A94000EC76E200EC66E9E96C69E2C
:10472000C50EC96EFF0E9EB602D0E82EFCD79E962F
:10473000C69E000EC96EFF0E9EB602D0E82EFCD7B4
:10474000C9CF00F69E96C69E000EC96EFF0E9EB69D
:1047500002D0E82EFCD7C9CF01F68A841200000EE1
:10476000C76E200EC66E8A949E96C69EC80EC96EEF
:10477000FF0E9EB602D0E82EFCD79E96C69E000E77
:10478000C96EFF0E9EB602D0E82EFCD7C9CF02F646
:104790009E96C69E000EC96EFF0E9EB602D0E82EF3
:1047A000FCD7C9CF03F68A848A949E96C69ECA0E09
:1047B000C96EFF0E9EB602D0E82EFCD79E96C69E0E
:1047C000000EC96EFF0E9EB602D0E82EFCD7C9CFF0
:1047D00004F69E96C69E000EC96EFF0E9EB602D0CF
:1047E000E82EFCD7C9CF05F68A848A949E96C69E89
:1047F000CC0EC96EFF0E9EB602D0E82EFCD79E9658
:10480000C69E000EC96EFF0E9EB602D0E82EFCD7E3
:10481000C9CF06F69E96C69E000EC96EFF0E9EB6C6
:1048200002D0E82EFCD7C9CF07F68A841200000E0A
:10483000C76E200EC66E8A949E96C69EE80EC96EFE
:10484000FF0E9EB602D0E82EFCD79E96C69E000EA6
:10485000C96EFF0E9EB602D0E82EFCD7C9CF08F66F
:104860009E96C69E000EC96EFF0E9EB602D0E82E22
:10487000FCD7C9CF09F68A848A949E96C69EEA0E12
:10488000C96EFF0E9EB602D0E82EFCD79E96C69E3D
:10489000000EC96EFF0E9EB602D0E82EFCD7C9CF1F
:1048A0000AF69E96C69E000EC96EFF0E9EB602D0F8
:1048B000E82EFCD7C9CF0BF68A848A949E96C69EB2
:1048C000EC0EC96EFF0E9EB602D0E82EFCD79E9667
:1048D000C69E000EC96EFF0E9EB602D0E82EFCD713
:1048E000C9CF0CF69E96C69E000EC96EFF0E9EB6F0
:1048F00002D0E82EFCD7C9CF0DF68A841200000E34
:10490000C76E200EC66E8A949E96C69E240EC96EF1
:10491000FF0E9EB602D0E82EFCD79E96C69EE40EF1
:10492000C96EFF0E9EB602D0E82EFCD78A848A9408
:104930009E96C69E200EC96EFF0E9EB602D0E82E31
:10494000FCD79E96C69E5F0EC96EFF0E9EB602D025
:10495000E82EFCD78A848A949E96C69E210EC96E44
:10496000FF0E9EB602D0E82EFCD79E96C69EC00EC5
:10497000C96EFF0E9EB602D0E82EFCD78A848A94B8
:104980009E96C69E260EC96EFF0E9EB602D0E82EDB
:10499000FCD79E96C69E000EC96EFF0E9EB602D034
:1049A000E82EFCD78A8412008984000EC76E220E7E
:1049B000C66E9E96C69E000EC96EFF0E9EB602D0B3
:1049C000E82EFCD79E96C69E000EC96EFF0E9EB6C0
:1049D00002D0E82EFCD7C9CFABF59E96C69E000E3E
:1049E000C96EFF0E9EB602D0E82EFCD7C9CFACF53B
:1049F0009E96C69E000EC96EFF0E9EB602D0E82E91
:104A0000FCD7C9CFADF59E96C69E000EC96EFF0EAF
:104A10009EB602D0E82EFCD7C9CFAEF59E96C69EB4
:104A2000000EC96EFF0E9EB602D0E82EFCD7C9CF8D
:104A3000AFF59E96C69E000EC96EFF0E9EB602D0C2
:104A4000E82EFCD7C9CFB0F59E96C69E000EC96E63
:104A5000FF0E9EB602D0E82EFCD7C9CFB1F58994DF
:104A600087EC27F012008984000EC76E220EC66EF6
:104A70009E96C69E800EC96EFF0E9EB602D0E82E90
:104A8000FCD79E96C69EABC5C9FFFF0E9EB602D050
:104A9000E82EFCD79E96C69EACC5C9FFFF0E9EB6FB
:104AA00002D0E82EFCD79E96C69EADC5C9FFFF0E6C
:104AB0009EB602D0E82EFCD79E96C69EAEC5C9FF14
:104AC000FF0E9EB602D0E82EFCD79E96C69EAFC5BE
:104AD000C9FFFF0E9EB602D0E82EFCD79E96C69E5A
:104AE000B0C5C9FFFF0E9EB602D0E82EFCD79E9639
:104AF000C69EB1C5C9FFFF0E9EB602D0E82EFCD7F8
:104B0000899487EC27F012008984000EC76E220E6C
:104B1000C66E9E96C69E070EC96EFF0E9EB602D04A
:104B2000E82EFCD79E96C69E000EC96EFF0E9EB65E
:104B300002D0E82EFCD7C9CFABF59E96C69E000EDC
:104B4000C96EFF0E9EB602D0E82EFCD7C9CFACF5D9
:104B50009E96C69E000EC96EFF0E9EB602D0E82E2F
:104B6000FCD7C9CFADF59E96C69E000EC96EFF0E4E
:104B70009EB602D0E82EFCD7C9CFAEF5899487EC5B
:104B800027F08984000EC76E220EC66E9E96C69EC2
:104B90000F0EC96EFF0E9EB602D0E82EFCD79E9671
:104BA000C69E000EC96EFF0E9EB602D0E82EFCD740
:104BB000C9CFB3F5899487EC27F012008984000EE1
:104BC000C76E220EC66E9E96C69E870EC96EFF0EDB
:104BD0009EB602D0E82EFCD79E96C69EABC5C9FFF6
:104BE000FF0E9EB602D0E82EFCD79E96C69EACC5A0
:104BF000C9FFFF0E9EB602D0E82EFCD79E96C69E39
:104C0000ADC5C9FFFF0E9EB602D0E82EFCD79E961A
:104C1000C69EAEC5C9FFFF0E9EB602D0E82EFCD7D9
:104C2000899487EC27F089849E96C69E8F0EC96E64
:104C3000FF0E9EB602D0E82EFCD79E96C69EB3C548
:104C4000C9FFFF0E9EB602D0E82EFCD7899487ECF0
:104C500027F012008984000EC76E220EC66E9E9643
:104C6000C69E870EC96EFF0E9EB602D0E82EFCD7F8
:104C70009E96C69E000EC96EFF0E9EB602D0E82E0E
:104C8000FCD79E96C69E800EC96EFF0E9EB602D0C1
:104C9000E82EFCD79E96C69E800EC96EFF0E9EB66D
:104CA00002D0E82EFCD79E96C69E800EC96EFF0EDF
:104CB0009EB602D0E82EFCD7899487EC27F0898431
:104CC0009E96C69E8F0EC96EFF0E9EB602D0E82E2F
:104CD000FCD79E96C69E010EC96EFF0E9EB602D0F0
:104CE000E82EFCD7899487EC27F012008984000E07
:104CF000C76E220EC66E9E96C69E870EC96EFF0EAA
:104D00009EB602D0E82EFCD79E96C69E000EC96EB7
:104D1000FF0E9EB602D0E82EFCD79E96C69E000ED1
:104D2000C96EFF0E9EB602D0E82EFCD79E96C69E98
:104D3000800EC96EFF0E9EB602D0E82EFCD79E965E
:104D4000C69E800EC96EFF0E9EB602D0E82EFCD71E
:104D5000899487EC27F089849E96C69E8F0EC96E33
:104D6000FF0E9EB602D0E82EFCD79E96C69E010E80
:104D7000C96EFF0E9EB602D0E82EFCD7899487EC50
:104D800027F012008984000EC76E220EC66E9E9612
:104D9000C69E8F0EC96EFF0E9EB602D0E82EFCD7BF
:104DA00087EC27F09E96C69E810EC96EFF0E9EB6BA
:104DB00002D0E82EFCD7899487EC27F08984000E76
:104DC000C76E220EC66E9E96C69E8F0EC96EFF0ED1
:104DD0009EB602D0E82EFCD787EC27F09E96C69EA2
:104DE000010EC96EFF0E9EB602D0E82EFCD7899444
:104DF00087EC27F089849E96C69E910EC96EFF0EA1
:104E00009EB602D0E82EFCD787EC27F09E96C69E71
:104E1000A50EC96EFF0E9EB602D0E82EFCD789946F
:104E200087EC27F012008984000EC76E220EC66E32
:104E30009E96C69E8F0EC96EFF0E9EB602D0E82EBD
:104E4000FCD787EC27F09E96C69E810EC96EFF0E9A
:104E50009EB602D0E82EFCD7899487EC27F012008A
:104E60008984000EC76E220EC66E9E96C69E8F0E59
:104E7000C96EFF0E9EB602D0E82EFCD787EC27F055
:104E80009E96C69E010EC96EFF0E9EB602D0E82EFB
:104E9000FCD7899487EC27F012008984000EC76E36
:104EA000220EC66E9E96C69E910EC96EFF0E9EB6CF
:104EB00002D0E82EFCD787EC27F09E96C69EA50E62
:104EC000C96EFF0E9EB602D0E82EFCD7899487ECFF
:104ED00027F012008984000EC76E220EC66E9E96C1
:104EE000C69E910EC96EFF0E9EB602D0E82EFCD76C
:104EF00087EC27F09E96C69E000EC96EFF0E9EB6EA
:104F000002D0E82EFCD7899487EC27F01200050E1A
:104F1000E82EFED712000501256B266B276B286B48
:104F2000899A400EC76E200EC66E9E96C69E030ED0
:104F3000C96EFF0E9EB602D0E82EFCD79E96C69E86
:104F400027C5C9FFFF0E9EB602D0E82EFCD79E965D
:104F5000C69E26C5C9FFFF0E9EB602D0E82EFCD71E
:104F60009E96C69E25C5C9FFFF0E9EB602D0E82EAE
:104F7000FCD79E96C69EC952FF0E9EB602D0E82E62
:104F8000FCD7898A0F01C950FF0A01E1120005010F
:104F90002E51130A05E005012E51170A0CE01200EC
:104FA0000501F00E256FFF0E266F0F0E276F000E06
:104FB000286FE4EF27F00501F00E256FFF0E266F36
:104FC000FF0E276F000E286F899A400EC76E200EC5
:104FD000C66E9E96C69E030EC96EFF0E9EB602D08A
:104FE000E82EFCD79E96C69E27C5C9FFFF0E9EB62B
:104FF00002D0E82EFCD79E96C69E26C5C9FFFF0E9E
:105000009EB602D0E82EFCD79E96C69E25C5C9FF47
:10501000FF0E9EB602D0E82EFCD79E96C69EC952C1
:10502000FF0E9EB602D0E82EFCD7898A0F01C95028
:10503000FF0A1EE005012E51130A05E005012E515D
:10504000170A0CE012000501000E256F000E266FF6
:10505000100E276F000E286FE4EF27F00501000EF9
:10506000256F000E266F000E276F010E286F1200AD
:105070000501256B266B276B286B05012E51130A42
:1050800005E005012E51170A0CE012000501000E83
:10509000216F000E226F040E236F000E246F5AEF53
:1050A00028F00501000E216F000E226F800E236F85
:1050B000000E246F21C500F122C501F123C502F1C4
:1050C00024C503F125C504F126C505F127C506F160
:1050D00028C507F191EC20F000C125F501C126F5A6
:1050E00002C127F503C128F5899A400EC76E200E2C
:1050F000C66E9E96C69E030EC96EFF0E9EB602D069
:10510000E82EFCD79E96C69E27C5C9FFFF0E9EB609
:1051100002D0E82EFCD79E96C69E26C5C9FFFF0E7C
:105120009EB602D0E82EFCD79E96C69E25C5C9FF26
:10513000FF0E9EB602D0E82EFCD79E96C69EC952A0
:10514000FF0E9EB602D0E82EFCD7898AC950FF0A0E
:1051500008E104C125F505C126F506C127F507C1FB
:1051600028F5D890050124332333223321332151EC
:10517000F00B216F2167C4EF28F02267C4EF28F0FD
:105180002367C4EF28F024675AEF28F00501100EBA
:105190002527E86A2623E86A2723E86A28231200DD
:1051A000E86A05012E51130A06E005012E51170A7F
:1051B0000BE0020E120005012851000A03E12751FD
:1051C000F00B07E0010E120005012851000A01E072
:1051D000010E120029C500F12AC501F12BC502F10B
:1051E0002CC503F125C504F126C505F127C506F137
:1051F00028C507F120EC22F003BF1200D0EC28F004
:105200005FE1899A400EC76E200EC66E9E96C69EBE
:10521000060EC96EFF0E9EB602D0E82EFCD7898A14
:10522000899A9E96C69E020EC96EFF0E9EB602D049
:10523000E82EFCD79E96C69E27C5C9FFFF0E9EB6D8
:1052400002D0E82EFCD79E96C69E26C5C9FFFF0E4B
:105250009EB602D0E82EFCD79E96C69E25C5C9FFF5
:10526000FF0E9EB602D0E82EFCD79E96C69E000E7C
:10527000C96EFF0E9EB602D0E82EFCD7898A899AA5
:105280009E96C69E050EC96EFF0E9EB602D0E82EF3
:10529000FCD79E96C69EC952FF0E9EB602D0E82E3F
:1052A000FCD7C9B049EF29F0898A0501100E2527DE
:1052B000E86A2623E86A2723E86A2823EAEF28F029
:1052C0001200899A400EC76E200EC66E9E96C69E2C
:1052D000060EC96EFF0E9EB602D0E82EFCD7898A54
:1052E000899A9E96C69EC70EC96EFF0E9EB602D0C4
:1052F000E82EFCD7898A0501256B266B276B286B66
:105300001200899A400EC76E200EC66E9E96C69EEB
:10531000050EC96EFF0E9EB602D0E82EFCD79E96F3
:10532000C69EC952FF0E9EB602D0E82EFCD7C9CF4A
:1053300033F5898A1200899A400EC76E200EC66E18
:105340009E96C69EB90EC96EFF0E9EB602D0E82E7E
:10535000FCD7898A1200899A400EC76E200EC66E4D
:105360009E96C69EAB0EC96EFF0E9EB602D0E82E6C
:10537000FCD7898AFF0EE82EFED71200D0EC28F069
:10538000D8A41200899A400EC76E200EC66E9E9653
:10539000C69E030EC96EFF0E9EB602D0E82EFCD745
:1053A0009E96C69E27C5C9FFFF0E9EB602D0E82E68
:1053B000FCD79E96C69E26C5C9FFFF0E9EB602D09C
:1053C000E82EFCD79E96C69E25C5C9FFFF0E9EB649
:1053D00002D0E82EFCD79E96C69EC952FF0E9EB6FE
:1053E00002D0E82EFCD7898A0F01C950FF0AD8A441
:1053F000BDEF2AF00501FE0E336F0501000E336F7D
:10540000D4EC24F0ABC534F5ACC535F5ADC536F5F7
:10541000AEC537F5AFC538F5B0C539F5B1C53AF504
:105420000784B6C166F1B7C167F1B8C168F1B9C107
:1054300069F14BC14FF14CC150F14DC151F14EC119
:1054400052F157C159F158C15AF1079492EC18F032
:1054500000C13BF501C13CF502C13DF503C13EF57C
:1054600005015D673BEF2AF05E673BEF2AF05F675F
:105470003BEF2AF060673FEF2AF04DEF2AF05DC561
:1054800004F15EC505F15FC506F160C507F10101D4
:1054900020EC22F003BFBDEF2AF059C13FF55AC1FD
:1054A00040F5B5C541F5B6C542F50501100E326FA0
:1054B000899A400EC76E200EC66E9E96C69E060E38
:1054C000C96EFF0E9EB602D0E82EFCD7898A899A53
:1054D0009E96C69E020EC96EFF0E9EB602D0E82EA4
:1054E000FCD79E96C69E27C5C9FFFF0E9EB602D06A
:1054F000E82EFCD79E96C69E26C5C9FFFF0E9EB617
:1055000002D0E82EFCD79E96C69E25C5C9FFFF0E89
:105510009EB602D0E82EFCD725EE33F0322F02D013
:105520009DEF2AF09E96C69EDECFC9FFFF0E9EB667
:1055300002D0E82EFCD78EEF2AF0898A899A9E96AF
:10554000C69E050EC96EFF0E9EB602D0E82EFCD791
:105550009E96C69EC952FF0E9EB602D0E82EFCD77C
:10556000C9B0A8EF2AF0898A0501100E2527E86A3C
:105570002623E86A2723E86A2823120021C500F1C0
:1055800022C501F123C502F124C503F1899A400E19
:10559000C76E200EC66E9E96C69E0B0EC96EFF0E7F
:1055A0009EB602D0E82EFCD79E96C69E02C1C9FFC9
:1055B000FF0E9EB602D0E82EFCD79E96C69E01C175
:1055C000C9FFFF0E9EB602D0E82EFCD79E96C69E5F
:1055D00000C1C9FFFF0E9EB602D0E82EFCD79E96F2
:1055E000C69EC952FF0E9EB602D0E82EFCD725EE0D
:1055F00033F00501100E326F9E96C69EC952FF0E03
:105600009EB602D0E82EFCD7C9CFDEFF322FFCEFCA
:105610002AF0898A1200899A400EC76E200EC66E43
:105620009E96C69E900EC96EFF0E9EB602D0E82EC4
:10563000FCD79E96C69E000EC96EFF0E9EB602D087
:10564000E82EFCD79E96C69E000EC96EFF0E9EB633
:1056500002D0E82EFCD79E96C69E000EC96EFF0EA5
:105660009EB602D0E82EFCD79E96C69EC952FF0E6B
:105670009EB602D0E82EFCD7C9CF2DF59E96C69EC9
:10568000C952FF0E9EB602D0E82EFCD7C9CF2EF528
:10569000898A12000CEC21F0B5C5E8FFD70802E3B7
:1056A0000CEC21F0B5C5E8FFC80802E30CEC21F0D2
:1056B000B5C5E8FFB90802E30CEC21F0B5C5E8FF79
:1056C000AA0802E30CEC21F0B5C5E8FF9B0802E351
:1056D0000CEC21F084EC25F09BEC29F0F29CF29E7E
:1056E0008B94899CC69AC2908A848A969482948C60
:1056F000720ED36ED3A4FED789968A909390FF0E34
:10570000E8CF00F0E82EFED7002EFCD78150F294AF
:10571000F29A9E909D909E929D92F298F292F290B3
:08572000F286F28E0300FF0087
:10BF0000E844F926000C160C2B0C3F0C520C640C68
:10BF1000760C860C960CA50CB30CC10CCF0CDC0C6B
:06BF2000E80CF40C000C1B
:00000001FF
